:020000040000FA
:060000000219FD020310CD
:030013000204FFE5
:03001B0002008D53
:03002B000202D5F9
:03005B0002050E8D
:030073000202FD89
:100080000406080C10182030406080A0C0C2AFC227
:10009000A853E6EFC28E856B8BC0D0D2D3C0E0C030
:1000A000F0C2CAA8CCA9CDD2CAD2AF758A00C3E823
:1000B000956CF8E9956DF9C3E913F9E813F8E5666D
:1000C0006007C3E913F9E813F8E97025E8956E4075
:1000D00020956E501CE582B410177C007B007A00DE
:1000E0007908900000A86AE5667004C3E813F80177
:1000F000FA900000D2A8D2AA61BAE0FDC39CC398CE
:1001000040EF98EB33FB0582E0FCC39DC39840E1D0
:1001100098EB33FB0582E0FDC39CC39840D398EB7A
:1001200033FB0582E0FCC39DC39840C598EB33FBCD
:100130000582E0FDC39CC39840B798EB33FB058272
:10014000E0FCC39DC39840A998EB33FB0582E0FD1A
:10015000C39CC398409B98EB33FB0582E0FCC39D96
:10016000C398408D98EB33FB05822175900000D237
:10017000A8D2AA61BAE0FDC39CC39840EF98EA33C5
:10018000FA0582E0FCC39DC39840E198EA33FA0582
:1001900082E0FDC39CC39840D398EA33FA0582E01D
:1001A000FCC39DC39840C598EA33FA0582E0FDC3BD
:1001B0009CC39840B798EA33FA0582E0FCC39DC31C
:1001C0009840A998EA33FA0582E0FDC39CC39840A1
:1001D0009B98EA33FA0582E0FCC39DC398408D9852
:1001E000EA33FA0582EBC46B6A54F0F9EAC454F0BE
:1001F000C3996009900000D2A8D2AA61BAEBF4C4F6
:1002000054F0F9EAF4C4540F49FAEBF4C4540FFB68
:10021000C3EAF99460FAEB9400FB5020C3E97B0039
:100220007A0079006016C3135006F9C39552600A2C
:10023000E9F552755300790080020553303A27C31F
:10024000EA94D0F8EB9407F9400BE8FAE9FB203583
:1002500009D235415A303502C235203902B235C390
:10026000EA33FAEB33FBEB2B3B3BF9C3EB13FBEA33
:1002700013FAEA29FAEB3400FB30E3047AFF7BFF40
:10028000E5255403601B202A18E55D33F9EB700760
:10029000C3E99A4002E9FAE53CC4332AFAEB340098
:1002A000FBC3EA33C4540FF8EB33C454F048F8707E
:1002B00005EA60027801C3EB13FBEA13FA90000031
:1002C000D2A8D2AAE52260021522819E900000D217
:1002D000A8D2AA61BAC0D0C0E0C2CF0541E5236070
:1002E000021523C3E554600575550041F8E5552412
:1002F00001F55550037555FFD0E0D0D032C2AF5351
:10030000E67F7592FA7593FFC22053917FD2AF3288
:10031000C0E0E58A303408856B8BF0A3D0E032D0A2
:10032000E0C2AF53E6EFC0D0C0E0C0F0D2D3D2AF4E
:100330005388EFA88AA98C758A00758C00438810B1
:1003400030331FE8C4540FFAE9C454F04AFAC31317
:100350002AFAC3E833F8E933F9E82AFAE93403FB67
:1003600061AB30320FC3E833E933FAE82AFAE934F3
:1003700000FB61AB303115E875F056A4AAF0E975C1
:10038000F056A42AFAC5F03400FB61ABE875F02BF7
:10039000A4AAF0E975F02BA42AFAC5F03400C3131F
:1003A000FBEA13FAC3EB13FBEA13FAC3EB9409500D
:1003B00009C3EA949AEB940350160522E5227002D1
:1003C0001522C3E5229432500281F275540081F562
:1003D000E522600215223036067C007D0461EAAC1D
:1003E00031AD32303A04AC33AD34C3EA9CFAEB9D04
:1003F000FB9208AE60AF61303A425007203509D217
:10040000358108303502C235303504AE62AF632025
:100410003902B235C3EA33FAEB33FBA208500AEAD9
:10042000F42401FAEBF43400FBC3EA9428FAEB94C9
:1004300000FB501478007A007B008148A208500825
:1004400078007A007B00819EE52554036019202AFC
:1004500016E55DF9EB7007C3E99A4002E9FAE53C5D
:10046000C42AFAEB3400FBEA8EF0A4F9AAF0EB8E72
:10047000F0A42AFAC5F03400FBC3EB13FDEA13F82D
:100480000FEF146004C3E833F8C3E933EA33FAEB3F
:1004900033FBDFEDEB30E20678FF7AFF7B03885415
:1004A000D230E86003755500C3E55BFC955C400203
:1004B000AC5CC3EC95545008EC75F004A4FAABF0B6
:1004C000EAF4F8EBF45403F9C3E89419FAE9940058
:1004D000FB50047A007B00885689578A588B5975DF
:1004E000230AD0F0D0E0D0D053F7DF43F74043E603
:1004F000103275230AD0F0D0E0D0D043E61032C2DB
:10050000AAD28EC2CA85CC6C85CD6DD2CA32C2AF9A
:10051000C0D0C0E0D2D3A8F9E55A30E10AE5FA200C
:10052000E13520E032A12FE5FA30E12B20E028C3AD
:10053000E55713F8E55613F5FB88FCC3E55913F8A6
:10054000E55813F5E988EA85575A53F7BFD2A83022
:100550003402D2AA53E6EF53F7DFD0E0D0D0D2AFC7
:10056000327901801479038010790A800C791E8019
:10057000087964800479C880007817E4D5E0FDD854
:10058000FAD9F62278FF20282879A1E76023E548E8
:10059000601F74FF8548F084853FF030290375F0B3
:1005A00005A4F8C5F0600278FFC3E8955D5002A885
:1005B0005D885C22C3E54794E4E5489400E55C501F
:1005C0000314A1C5046002F55C2275E89022055E63
:1005D000C3E55E9408405330EDF4A8BDA9BE755E36
:1005E00000E9FA79A0E76041EA7006E55F601880EB
:1005F0000CC3E8955F600EE55F5005600A14800744
:100600000460FA8002E55FF55FC39569401B755B86
:10061000C0C394044013755B80C39404400B755BA6
:1006200040C394044003755B0022E55B2410500234
:1006300074FFF55B22743279A687F0A4C5F0A2F7A7
:1006400033F55D227547007548F022C2AFC2CAA8D3
:10065000CCA9CDAA4130CF010AD2CAD2AFAB42ACAD
:100660004388428943C3E89BF8E99C202808F93075
:100670002C02E15BC1B4AD448A44F9EA9DFA6006FC
:1006800078FF79FFC199AE45AF468B458C46A842AD
:10069000A943C3E89EF8E99FF9C3E54813FBE54782
:1006A00013FAE82AF547E93BF54850067547FF7508
:1006B00048FFE101AA47AB48AC47AD487E047F0242
:1006C000C3EB9404400D1E1FC3EB94084005202982
:1006D000021E1FC3ED13FDEC13FCDEF7C3EA9CFA08
:1006E000EB9DFBEF6009C3E913F9E813F8DFF7EAC4
:1006F00028FAEB39FB8A478B4850067BFF8B478BE8
:1007000048C3EB94025002D22C3028047F03E12C22
:100710007892E6FFC3E53D948240110FC3E53D9416
:10072000A040010FC3EF940640027F057E02E5481A
:10073000C4540FF9E548C454F0F8E547C4540F28F1
:10074000F8C3E89EFAE99400FB4009C3EA9401EB80
:10075000940050047A01E4FB0207A7AA47AB48EBD8
:10076000C4FEEAC4540F4EFCC3EA9CFAEB9400FBAF
:10077000C3E813C313F8EA28FAEB3400FB8A478B6B
:1007800048C3EB94024002C22C7802EBC4FE7B000B
:10079000EAC4540F4EFAC3EA98FA4005C3940150D4
:1007A000027A017892E6FF302002E1A7854E928519
:1007B0004F93D22043E680C3E49AF8E49BF9302CAF
:1007C00003020835E8FAE9FBD3E913FDE813FC88D6
:1007D0004E894FC3EF94036038EF20E00CE82CF80B
:1007E000E93DF9ECFAEDFB8013E828F8E939F9C3A3
:1007F000E82401F8E93400F97AFF7BFFC3EF9403A2
:10080000400F8A508B51884A894B8C4C8D4D020881
:100810006A885089518A4A8B4B8C4C8D4D302812F6
:100820007550F07551FF754CF0754DFF754EF075B4
:100830004FFF02086AE8FAD3E813FC884EC3EF942E
:10084000036021EF20E007E82CF8ECFA0155E828D6
:100850002401F87AFFC3EF940340098A50884A8C38
:100860004C02086A88508A4A8C4C302002016A7512
:100870003A02D22043E680E52554036034A847A914
:1008800048C3E913F9E813F8C3E913F9E813F8309A
:100890002804E92440F9C2AF53E67F759100C3E410
:1008A00098F594E499F595759104D22043E680D2A9
:1008B000AF22D221754900752000302B03752040EE
:1008C00001D0D221754900752040302B03752000DE
:1008D00078017901202C20E52554036002C221799A
:1008E00014E548C313700104F8C39414400278144B
:1008F000302804781B791B202010E549600C302833
:1009000003D53A04D222217711720549E5BF54403C
:10091000B52002216130280908C3E8994001180177
:10092000F720210A08C3E899400201D001F7C2214B
:1009300053E67F759100302C117594007595F8750C
:100940009104D22043E6800208D0E5487EFFC333FD
:100950004005C3334001FEC3E49E759400F5952124
:100960003FC3E5399401500201D030210201D0D8B3
:1009700002217501F7C222C2AF53E67F759100854F
:100980005094855195759104854A92854B93D22058
:1009900043E680D2AFE525540360072029020539DC
:1009A000801030220D202B0A20210715811581028D
:1009B00013772278003021027801E53D75F007A415
:1009C000F9E5F028F5F0E9A2F013A2F113A2F21371
:1009D000F53DC394785003753D78C3E53D953E40A1
:1009E0000CC285C286C28775D4FF75D50730200238
:1009F00021ED854C92854D93D22043E6802220380C
:100A000013C2AFC291D29075D47F75D503D2AF75A2
:100A1000AA5341F2C2AFC291D29275D4DF75D50606
:100A2000D2AF75AA5341F2203813C2AFC28775D432
:100A3000BF75D505D290D2AF75AA4341F2C2AFC2FD
:100A40008575D4BF75D505D292D2AF75AA6341F230
:100A5000203813C2AFC290D29275D4BF75D505D2DB
:100A6000AF75AA6341F2C2AFC292D29075D4BF757E
:100A7000D505D2AF75AA438079203813C2AFC2869C
:100A800075D4DF75D506D292D2AF75AA538063C2F2
:100A9000AFC28675D47F75D503D290D2AF75AA53F5
:100AA0008050203813C2AFC292D29175D4DF75D571
:100AB00006D2AF75AA43803AC2AFC290D29175D424
:100AC0007F75D503D2AF75AA638027203813C2AFD4
:100AD000C28575D47F75D503D291D2AF75AA6380D4
:100AE00011C2AFC28775D4DF75D506D291D2AF756A
:100AF000AA43227A147B7880127A107B8C800C7A3D
:100B00000D7BB480067A0B7BC88000E564D5E001DC
:100B1000227902E4C291D5E0FDD286D5E0FDC286FD
:100B2000D5E0FDD291D5E0FDE920E002D28530E0AC
:100B300002D287E564D5E0FDE920E002C28530E01D
:100B400002C2877496D5E0FDD9C9EAF8D5E0FDD890
:100B5000FBDBB8C29122C285C286C287C290C29115
:100B6000C29275D4FF75D50722788076FF0876FF8C
:100B70000876FF0876FF0876FF0876FF08760908F2
:100B800076FF087601788C76010876FF0876FF08F4
:100B900076FF0876FF0876FF0876030876FF08766A
:100BA000FF0876FF0876250876D008762808765064
:100BB0000876040876FF0876020876FF08767A0839
:100BC00076FF0876070876010876FF0876FF087634
:100BD0000008760022FA75F00CA4ABF0EAC333F8F3
:100BE000740133F9E8C333F8E933F9E8C32BF8E9C2
:100BF0003400F9227888E6C39403D23A5002C23A0C
:100C0000C238E630E102D238A23892397886E6144A
:100C10009000809378A6F67886E6F53FC39402505C
:100C200003753F02789CE6753EFFB40203753EA053
:100C3000B40303753E8278A0E6F8600674282409A0
:100C4000D8FCF5697896E671D588318932789EE6C8
:100C500071D5883389347897E671D58835893671AE
:100C600056223036117A007B007CFF7D007E009199
:100C7000C88B618A6022303A227896E6FA7B007847
:100C80009EE6FC7D00C3EA33FAEB33FBC3EC33FC96
:100C9000ED33FD7E0A91C88B638A627896303A0202
:100CA000789EE6FA7B007897E6FC7D007E00303A7D
:100CB00010C3EA33FAEB33FBC3EC33FCED33FD7EB8
:100CC0000A91C88B618A6022C3EC9EFCED9400FD02
:100CD000C3EC9AFCED9BFDC3EC9423ED940050040F
:100CE0007C237D00C3EC94FFED940140047CFF7DE8
:100CF000017BFF0B7A000AEA7009C3EC33FCED3389
:100D0000FD81F3EC8AF0A4AEF0ED8AF0A42E947C81
:100D100040E4EAF460DD22D236916212056D1205DC
:100D20006D7A007B007C10120565E5542AFA740088
:100D30003BFBDCF37C04C3EB13FBEA13FADCF7FFA9
:100D4000EB60027FFFC23691622278A5E6F9540378
:100D5000D2837002C283E9540CD2847002C284E947
:100D600054307000E954C070002275670075680047
:100D70007597DE7597AD7581C043FF8075EF067579
:100D8000A900715675800275F1FF75A4F87580028F
:100D900075D4FF75900075F20775A50775900075FD
:100DA000D50775A60175E34075E2027156E4F8F6C1
:100DB000D8FD71691213AC78988664753001C2AFA2
:100DC00012057551F312056D51F912056D51FF129F
:100DD000056DB14AC2AF75670075680078FA79FA97
:100DE000308107D9FBD8F7021C0071F49162789822
:100DF0008664715675E401758811758E04758909CC
:100E000075C80475910475D84075D90875F7817552
:100E10009E0375960275DA4275DB4275A82175E668
:100E20009075B80175BF8075AB0075D10C75BC5954
:100E300075BB1075E88075B201120561D2AF753CC3
:100E400000C230120575C231C232C233C23475528B
:100E500000752200120571C3E522940A5002E128B0
:100E6000D231752200120571C3E522940A5002E1C5
:100E700028C231D232752200120571C3E522940ACC
:100E80005002E12875E491758851758E017589AA23
:100E9000758C00758D00C2A9D2ABD2AA756BC075D6
:100EA0006A14756E50C232D23475220A12057175F9
:100EB0006A10C3E522940A755200755300406975A3
:100EC0008E0C756B80756A28756E2875220A12055E
:100ED00071756A20C3E522940A755200755300406B
:100EE00047758E0C756BC0756A14756E1475220A81
:100EF000120571756A10C3E522940A755200755384
:100F000000402575E401758811758E04758909D234
:100F1000A9C2ABC2AAC234D233752200120571C372
:100F2000E522940A4002A1D4120565203003020D87
:100F3000D4C2AF51F351F351F3D2AF12057520343F
:100F400003303A03020FE6120565788CE6C394017C
:100F50005002E1E6E530C394015002E1E67567A571
:100F60007568F17F02D2369162120571C2AFC23646
:100F70009162C3E554947FD2AF406B120561C2AF5A
:100F80007105D2AFDFDFB117C3EF7897F6120575A1
:100F90001214997F0AD2369162120571C2AFC2361D
:100FA0009162C3E554947FD2AF50E8120561C2AF9D
:100FB00051F312056951F3D2AFDFDAB117EF240311
:100FC0007896F6F87997E7C394234003985006E89B
:100FD00024237897F61205751213F31214C812051C
:100FE000719162020DD4756700756800120571C3B6
:100FF000E55494014002E13EC2AF71057105120B48
:1010000005D2AF120575753000E4F537F5380537B0
:10101000E537F4703F0538789AE67819146012784D
:101020003214600D787D14600878FA146003753806
:1010300000C3E53898401D120B561205611538752E
:10104000370078998664C2AF120B05D2AF789886C4
:1010500064120571120569E5237003020DD4C3E51E
:101060005294015014C3E554940140A2120571E555
:10107000237003020DD4021217C3E55294017017B6
:10108000C2AF120B5678998664120AF37898866478
:10109000D2AF1205714109C3E55294027017C2AF75
:1010A000120B5678998664120AF978988664D2AF42
:1010B0001205714109C3E55294037017C2AF120BB8
:1010C0005678998664120AFF78988664D2AF120522
:1010D000714109C3E55294047013C2AF120B5678E4
:1010E000998664120B05D2AF1205714109C3E5520E
:1010F00094057017C2AF120B5678998664120B05CF
:1011000078988664D2AF1205714109C3E5529407FD
:101110007019C3E55394095002015E7401303A021C
:1011200074037888F6C238C2394109C3E55294087D
:101130007019C3E55394095002015E7402303A02FB
:1011400074047888F6D238D2394109C3E55294093B
:101150007017C3E55394095002015E303A0BC3780F
:1011600088E69402F6C23A4109C3E552940A701621
:10117000C3E55394095002015E203A0A7888E624B8
:1011800002F6D23A4109C3E55294147025C3E553DF
:1011900094095002015EC2AF901A0B740093D2AF53
:1011A0007888F613C238C2394002D2384002D239A8
:1011B0008057C3E55294157038C3E5539409404FE6
:1011C000C2AF901A0B740093D2AFF8B80102740248
:1011D000B802027401B803027404B80402740378FC
:1011E00088F613C238C2394002D2384002D2398060
:1011F00018C3E552940C70117567A57568F1C3E5C5
:10120000539409400A71F3D2AF75520075530075BB
:101210006700756800015EC2AF120B56E4D2AFE4FE
:10122000F55EF524F525F53D755E0812056112059C
:10123000CA30EDFDA8BDA9BEE97001F8885F1205AE
:10124000CE755E08C2AF120635855D5B855D5CD2EA
:10125000AF303A07C238303502D238D2287539005B
:10126000120AA2120ACB12064412064B12064412AC
:10127000064B1206441208C21209B31209FE1206E6
:101280004B1208B2202C03120584302C031205B433
:101290001209B3120A2712064B1208C21209B3121E
:1012A0000A5012064B1208B21209B3120A7912063A
:1012B0004B1208C21209B3120AA212064B1205CA37
:1012C0001208B21209B3120ACB1205CE12064B3025
:1012D0002827855D5B79187A0CC3E53999400EC2E1
:1012E00028D2298A3B855D5B855D5C800CC3E55413
:1012F00094014003021275617F30291F202B1CE5E9
:101300003B147006C229D22A4175F53B203A07C327
:10131000E554940140030212758064753C00203A44
:101320000F78FA79A4E760027803C3E55598504F27
:10133000E523604B303A17203805203507800F3001
:101340003502800A202B07D22B855D5B41A578F002
:10135000302B05855D5B7820C3E548985003021269
:1013600075302B1BC22BC238303502D238D22975CA
:101370003B12855D5B4175053CE5546002618275F9
:101380003C00C2AF120B56752400752500D2AF1277
:101390000571120B5678A4E66006D290D291D292D3
:1013A000C3E53C94044003020DD40109901A0D7862
:1013B00020912CE520B4550AA3912CE520B4AA0273
:1013C00080137567A57568F1120B6971F375670075
:1013D000756800801D901A0378807B0A912CA30801
:1013E000DBFA901A0F788C7B1A912CA308DBFA9009
:1013F0001A2922C2AF916F914C901A00741091314A
:10140000A3743E9131A374219131901A0378807BAB
:101410000A9130A308DBFA901A0F788C7B1A91306E
:10142000A308DBFA91829160901A2922E493F622B4
:10143000E6438F01538FFDFFC3E583941C400122D7
:10144000EF8567B78568B7F0538FFE22438F02435D
:101450008F018567B78568B7901A0DF0538FFC220E
:10146000901A0D74559131901A0E74AA9131227A06
:101470003079D07820901A40912CE520F709A3DA32
:10148000F7227A3079D0901A40E7913109A3DAF93E
:10149000227C05120575DCFB22C2AF120AF3120A88
:1014A000F9120AFF120B05120569120AF3120AF962
:1014B000120AFF120B05120569120AF3120AF91239
:1014C0000AFF120B05D2AF22C2AF120B05120AFFA0
:1014D000120AF9120AF3120569120B05120AFF1219
:1014E0000AF9120AF3120569120B05120AFF120A11
:0714F000F9120AF3D2AF224A
:1019FD00020D6A103E21FFFFFFFFFFFF09FF01FFF0
:101A0D0055AA01FFFFFFFFFF03FFFFFF25D0285061
:0D1A1D0004FF02FF7AFF0701FFFF0000FF3A
:101A400023515F4C5F32352320202020202020208E
:101A500023424C48454C492445464D3842313023B9
:101A60002020202020202020202020202020202076
:101C0000C2AFC2D37597DE7597AD7581C075A90057
:101C100043FF80752438752503B1DB7529A5752A26
:101C2000F143F10253A4FDD28175D4FF75E3407DE9
:101C3000FA780379E67C10752200752300901DE880
:101C40007B06752498752501308102814820810822
:101C5000D8FBD9F9DCF781BA308108D8FBD9F9DC97
:101C6000F781BAB19BE493A3C39A6004DDC381BA40
:101C7000DBDBB18D600281317B08E493FAA3B16EA6
:101C8000DBF87A30B16E752200752300B18DEAFC65
:101C9000EBFDC3ED94FE400EB18D8A278B28ED300D
:101CA000E0048A828B83B18D7AC270D8C3ED94FE32
:101CB000601950CEBD0029EC600F7520007521FF22
:101CC000752900752A000200008100A827A92808AC
:101CD00009D804D90281DDB191EAF281D10D81A642
:101CE000C3ED94035051EDA2E092007AC5C3E582A2
:101CF0009400E583941C508C200010438F02438F86
:101D0000018529B7852AB7F0300027A827A9280818
:101D100009438F01538FFDD804D902A132C3E58353
:101D2000941C4003A3A117E28529B7852AB7F0A325
:101D3000A117538FFC81827AC1BD030CE493A3FAEF
:101D4000B152DCF8B14A81828184AA22AB23B16E00
:101D5000EBFAEA6222752608C3E52313F523E52290
:101D600013F52250066323A0632201D526EAB1DBD6
:101D7000B1DB75260AEAF4200102D281300102C2E9
:101D800081B1DBC3134002C201D526EB22B191EA37
:101D9000FB208102A191308102A196752608AE2414
:101DA000AF25C3EF13FFEE13FEB1DFB1DBC3EA13C0
:101DB0003081024480FA30E703632201C3E5231334
:101DC000F523E52213F52250066323A0632201D5F3
:101DD00026D9E52265236523F52222AE24AF250E00
:101DE0000FDEFEDFFCD20122424C48656C693437BD
:061DF0003164E8B10601B8
:00000001FF
